:02000000017B82
:20007B00758177900000E4F012043E12001B80FBC82581C822C92581C97A0022D083D082C7
:20009B00CF2581F581CFC082C08322CF2581F581CF22FBE0CB22FCE0FBA3E0CC22FAE0F925
:2000BB00A3E0CA2229F9E5F03AFA227C00CB30E7011CCB2275F00030E70215F022FDE493E8
:2000DB00A3FEE493A3FF4E7009E493FE740193FF800BE493A3B5050BE493B5F0068F838EDC
:2000FB0082E473A380D8FEEBA4FD8EF0ECA4FCEB8EF0A4C5F02C2DC5F022311B8EF0ED22B2
:20011B00C002C001AAF0F97E007D007F11C3E933F9EA33FADF08F5F0E9D001D00222ED339A
:20013B00FDEE33FEC3ED9BF5F0EE9C40E0ADF0FED380DBBB000122C333C5F033C5F0DBF7A2
:20015B0022BB000122C3C5F013C5F013DBF722240280022401C5F03400C5F022C3940280D7
:20017B0003C39401C5F09400C5F022317CF4C5F0F4C5F02245F07022042231DE4024801ACE
:20019B0031DE401E7014801A31DE400E7014800A31DE500E800431F26008E4F5F02231F2C4
:2001BB0060F8E4F5F0042231F240F780ED31F240F170E780ED31F240E170E780DD31F25093
:2001DB00E180D7C39BC5F09C20E70720D207C345F02220D2F9D322C5F0C39C7003E5F09B25
:2001FB0022900000E0A360EEE0FFA3E0A3CF2582F582EF3583F58380EBD28822D2A8D2AF6E
:20021B0022C2A822C0D0C0E0C0F0C000C001A2B34029E54A7006854FFA854EF9E54B700611
:20023B008551FC8550FB754900E54A554B600302037ED2A9D2B9D28C02037EE580F571A23A
:20025B00B6400302037EE574F8E571548068600302037EE571F572C2B6C2A2E5805440703C
:20027B000302035EE572541F2429F874FF700302037E14A2B440F6E580F573F6C2B7E57252
:20029B0054017003020353E57254026003020302E5725420F9E57454806002C2A0E902026A
:2002BB00F7754A0075FA0075F900E57203035403F54C8653188652E57454806002D2A0E9E8
:2002DB00E553C313F54FE55213F54EE54FC313F5F0E54E13F55685F057020353754A01863A
:2002FB00FA1886F9020353E572F9E57454806002C2A0E902034B754B0075FC0075FB00E5FA
:20031B007203035403F54D8655188654E57454806002D2A0E9E553C313F54FE55213F54E1B
:20033B00E54FC313F5F0E54E13F55885F0598008754B0186FC1886FB74FF602714A2B4503A
:20035B00F9802074FF601C14A2B440F9E572541F2409F8E6F573F580C2B774FF600514A29E
:1C037B00B450F97580FFD2B6D2B7D2A2C2AFD001D000D0F0D0E0D0D0D2AF3222F9
:05000300C2AF02021F64
:200399002275080075EF7075D80075FD1F22D2AFD2AED2DD22C2AEC2DD22C0D0C0E0C000DE
:2003B900E508232409F8A6D908A6DAE574703AE508B40235756B00E6540FF5671818E6541E
:2003D9000FF566956760224004F5688006E5679566F568740495685010E56C7005756C01D4
:1E03F9008007D2A1756C0080000508530807E5084420F5D8D000D0E0D0D0D2AF322209
:05003300C2AF0203B39F
:2004190022C28DC28C5389F0438901758A14758CFF22D2A9D2B9D28CD2AF22C2A9C28C2254
:0204390032226D
:05000B00C2AF02043940
:20043D002275C50075EB0075A80075E80075B80075F8007580FF75A0FF75B0FF75FD7F753D
:20045D00FA0075F90075FC0075FB00758780758920758DFD758BFD75884975985285F45F23
:20047D0085F35E85F26185F160E5A05480F5741209CEE4F576E57675F0007B207C001201F7
:20049D00C270090204C8E576057680E9E57679097A0075F0001200BFE4F7E57679297A0018
:2004BD0075F0001200BFE4F70204A3E4F5497401F54A7401F54BE4F54CE4F54DE4F5F0F5D1
:2004DD004E85F04F740175F000F54E85F04FE4F5F0F55685F057E4F5F0F55885F059120432
:2004FD001A12039A1203A7120214120217E5746003020513C2A1E4F5F0F55A85F05B1205CF
:20051D00F7E5746003020527C2A1E4F56C02051B22745575F000C0E0C0F0120CA515811505
:20053D0081744E75F000C0E0C0F0120CA515811581744275F000C0E0C0F0120CA5158115DE
:20055D0081744C75F000C0E0C0F0120CA515811581746B75F000C0E0C0F0120CA515811597
:20057D0081745675F000C0E0C0F0120CA515811581740D75F000C0E0C0F0120CA5158115CB
:20059D0081740A75F000C0E0C0F0120CA51581158122E56675F000F56D85F06E120907E57D
:2005BD006775F000F56D85F06E120907E56875F000F56D85F06E120907740A75F000C0E04F
:2005DD00C0F0120CA515811581740D75F000C0E0C0F0120CA51581158122E4F576E57675F9
:2005FD00F0007B087C001201C2700902066BE576057680E9E57675F0007B017C0012014ED6
:20061D002401C5F03400C5F079097A001200BFE71200CF7B087C0012014EC0E0C0F0E5765A
:20063D0075F0007B017C0012014E79097A001200BFD0F0D0E047F56D85F06E54FFC5F054BA
:20065D000FC5F0F56D85F06E12077E02060B742075F000C0E0C0F0120CA515811581E4F5B9
:20067D0076E57675F0007B027C001201C270090206EFE576057680E9E57675F0007B017CF2
:20069D000012014E2401C5F03400C5F079297A001200BFE71200CF7B087C0012014EC0E064
:2006BD00C0F0E57675F0007B017C0012014E79297A001200BFD0F0D0E047F56D85F06E5417
:2006DD00FFC5F0540FC5F0F56D85F06E12077E02068F742075F000C0E0C0F0120CA515811C
:2006FD001581E54A75F000F56D85F06E120907E54C75F000F56D85F06E120907E552855340
:20071D00F0F56D85F06E12077E742075F000C0E0C0F0120CA515811581E54B75F000F56DC1
:20073D0085F06E120907E54D75F000F56D85F06E120907E5548555F0F56D85F06E12077EBA
:20075D00740A75F000C0E0C0F0120CA515811581740D75F000C0E0C0F0120CA51581158135
:20077D0022E56D856EF05400C5F054F0C5F0F56F85F0707B0C7C0012015CF56F85F0707B84
:20079D000A7C0012019570030207BDE56F8570F02430C5F03400C5F0F56F85F0700207CF89
:2007BD00E56F8570F02437C5F03400C5F0F56F85F070E56F8570F0C0E0C0F0120CA51581BF
:2007DD001581E56D856EF05400C5F0540FC5F0F56F85F0707B087C0012015CF56F85F07010
:2007FD007B0A7C00120195700302081EE56F8570F02430C5F03400C5F0F56F85F07002081A
:20081D0030E56F8570F02437C5F03400C5F0F56F85F070E56F8570F0C0E0C0F0120CA515AF
:20083D00811581E56D856EF054F0C5F05400C5F0F56F85F0707B047C0012015CF56F85F0C1
:20085D00707B0A7C00120195700302087FE56F8570F02430C5F03400C5F0F56F85F07002F0
:20087D000891E56F8570F02437C5F03400C5F0F56F85F070E56F8570F0C0E0C0F0120CA5FB
:20089D0015811581E56D856EF0540FC5F05400C5F0F56F85F0707B0A7C0012019570030252
:2008BD0008D4E56F8570F02430C5F03400C5F0F56F85F0700208E6E56F8570F02437C5F092
:2008DD003400C5F0F56F85F070E56F8570F0C0E0C0F0120CA515811581742C75F000C0E0AC
:2008FD00C0F0120CA51581158122E56D856EF054F0C5F05400C5F0F56F85F0707B047C009F
:20091D0012015CF56F85F0707B0A7C001201957003020946E56F8570F02430C5F03400C55A
:20093D00F0F56F85F070020958E56F8570F02437C5F03400C5F0F56F85F070E56F8570F04A
:20095D00C0E0C0F0120CA515811581E56D856EF0540FC5F05400C5F0F56F85F0707B0A7C9B
:20097D0000120195700302099BE56F8570F02430C5F03400C5F0F56F85F0700209ADE56F19
:20099D008570F02437C5F03400C5F0F56F85F070E56F8570F0C0E0C0F0120CA5158115819B
:2009BD00742C75F000C0E0C0F0120CA51581158122C2A2E4F577E57775F0007B0A7C00122C
:2009DD0001C27009020A7FE577057780E9E475F001F56285F063E5628563F07B007C0C1245
:2009FD0001957003020A7975EF70E574700575D806800375D8048563FA8562F9D2DCE4F53A
:200A1D0076E57675F0007B057C001201C27009020A38E576057680E9020A2FE5F55480705D
:200A3D00FA85D95C85DA5DE55C855DF054FFC5F0540FC5F0F55C85F05DC39562C5F095636C
:200A5D00C5F0F56485F065E5628563F02408C5F03400C5F0F56285F0630209F3120A8802D5
:200A7D0009E4D2A275FA0075F90022744F75F000C0E0C0F0120CA515811581745575F00064
:200A9D00C0E0C0F0120CA515811581745475F000C0E0C0F0120CA515811581743075F00085
:200ABD00C0E0C0F0120CA515811581743D75F000C0E0C0F0120CA515811581E5628563F066
:200ADD00F56D85F06E12077E742075F000C0E0C0F0120CA515811581744975F000C0E0C063
:200AFD00F0120CA515811581744E75F000C0E0C0F0120CA515811581743075F000C0E0C02B
:200B1D00F0120CA515811581743D75F000C0E0C0F0120CA515811581E55C855DF0F56D858A
:200B3D00F06E12077E742075F000C0E0C0F0120CA515811581744375F000C0E0C0F0120CE1
:200B5D00A515811581744175F000C0E0C0F0120CA515811581744C75F000C0E0C0F0120CBB
:200B7D00A515811581743D75F000C0E0C0F0120CA515811581E5648565F0C0E0C0F0120CA1
:200B9D00C515811581F56D85F06E12077E742075F000C0E0C0F0120CA51581158174477503
:200BBD00F000C0E0C0F0120CA515811581744175F000C0E0C0F0120CA5158115817449755E
:200BDD00F000C0E0C0F0120CA515811581744E75F000C0E0C0F0120CA515811581743D753D
:200BFD00F000C0E0C0F0120CA515811581E55E855FF0F56D85F06E12077E744F75F000C0CE
:200C1D00E0C0F0120CA515811581744675F000C0E0C0F0120CA515811581745375F000C0EE
:200C3D00E0C0F0120CA515811581745475F000C0E0C0F0120CA515811581743D75F000C0D6
:200C5D00E0C0F0120CA515811581E5608561F0F56D85F06E12077E742075F000C0E0C0F0B8
:200C7D00120CA515811581740A75F000C0E0C0F0120CA515811581740D75F000C0E0C0F010
:200C9D00120CA5158115812278FB12008BE63099FDC299F5992274FFF5F030980A3098FD70
:200CBD00C298E59975F0002278FB12008BE60886F030F73A02018678F912008B8603088635
:200CDD0004088605088606ED8EF01201DE401CED8EF02278F912008B8603088604088605CB
:200CFD00088606ED8EF01201DE40E4EB8CF02278FB12008B860308860485FEF0E5017F0037
:1A0D1D001201C2600575F001E422EF0FF5F0A41201C270F6EF1475F00022CA
:00000001FF
